:020000040000FA
:1000000083160510851486018312C33086000510FF
:10001000FF308E00C32099200C08FA3C03193028C9
:1000200099200C08AA3C0319302899200C08003CA0
:1000300003193028F0308E00C32099200C08FA3CB8
:1000400003193028EB308E00C32099200C0890084B
:1000500099200C08910899200C0892084C2022281D
:1000600030280000080005309500950B3528080061
:100070000000000000000000000000000000000080
:100080000000000000000000000000000000000070
:10009000000000000000080010188610101C8614D4
:1000A00090180610901C06141008C039031D080093
:1000B0001108FF39031D61201208FF39031D642058
:1000C0000800101E67287228901E88287D28382076
:1000D0000616382086163820061238208612910B14
:1000E0006728080038208616382006163820861221
:1000F00038200612910F7228080038200615382083
:1001000086153820061138208611920F7D280800A8
:10011000382086153820061538208611382006111B
:10012000920B88280800051893280800051C9628BB
:1001300008008C01831605143120312083128F01B1
:10014000051CAA280F08003C031CBD2831201030D4
:100150008F07A0288518BD2896208F018F0A93202D
:100160008C0C8C1385188C17962008300F02031CFA
:10017000AE28932096209320962083160510831294
:100180000510382008008316851083128510312051
:100190008316051483128F01051CDD288D018D0A3D
:1001A0003120051CDD2810300D02031CCF288F0ADA
:1001B0000F08003C031CFA28CC288D018F018F0A00
:1001C0000E18E4288510E62885148D0A8E0C9620DA
:1001D000932008300F02031CDF280D1C85140D1816
:1001E0008510962093208316851483128518F6288F
:1001F00093209620831605108312051038200800DE
:02400E00F33F7E
:00000001FF
